:100000000C9465040C9482040C9482040C94820475
:100010000C9482040C9482040C9482040C94650960
:100020000C9482040C9482040C94470C0C9482046B
:100030000C9482040C94FB070C942A080C94820400
:100040000C9482040C9482040C9482040C94820418
:100050000C948204750677067E06C406F706F7063A
:10006000F706F706F706F706F706F706F706F706A8
:10007000F7067905F706EF057705F205AD05720677
:10008000B505C5057905EB06F706F706F706CD05B4
:10009000FA0620065A06E405E905C805EC0511062E
:1000A000CB0546064E065D06F706F706F706F70689
:1000B000F706F706F706EF05F706F205AD05720637
:1000C000B505C5057905EB06F706F706F706CD0574
:1000D000FA0620065A06E405E905C805EC051106EE
:1000E000CB0546064E065D06004080C0105090D0FD
:1000F0002060A0E03070B0F0044484C4145494D460
:100100002464A4E43474B4F4084888C8185898D80F
:100110002868A8E83878B8F80C4C8CCC1C5C9CDCBF
:100120002C6CACEC3C7CBCFC014181C1115191D1E7
:100130002161A1E13171B1F1054585C5155595D50F
:100140002565A5E53575B5F5094989C9195999D9BF
:100150002969A9E93979B9F90D4D8DCD1D5D9DDD6F
:100160002D6DADED3D7DBDFD024282C2125292D297
:100170002262A2E23272B2F2064686C6165696D6BF
:100180002666A6E63676B6F60A4A8ACA1A5A9ADA6F
:100190002A6AAAEA3A7ABAFA0E4E8ECE1E5E9EDE1F
:1001A0002E6EAEEE3E7EBEFE034383C3135393D347
:1001B0002363A3E33373B3F3074787C7175797D76F
:1001C0002767A7E73777B7F70B4B8BCB1B5B9BDB1F
:1001D0002B6BABEB3B7BBBFB0F4F8FCF1F5F9FDFCF
:1001E0002F6FAFEF3F7FBFFF76322E350A0053658A
:1001F0006C662D54657374204572726F723A2030AC
:100200006200496E697469616C697A6564210A00EB
:10021000203D3E204E6F20616E73776572206672BE
:100220006F6D20417564696F210A00203D3E204EAC
:100230006F20616E737765722066726F6D204D65F9
:100240006D6F7279210A00203D3E2043616E277454
:1002500020777269746520746F204D656D6F7279B7
:10026000210A00286429656C6574652C202867299B
:10027000657420616E696D732C2028732965742064
:10028000616E696D732C20287629657273696F6EB3
:100290000A00287429696D652C2028612975646914
:1002A0006F2C202863296F756E742C2028782943C1
:1002B0007573746F6D20636F756E740A00287929E9
:1002C0005365742061206672616D652C2073696DC1
:1002D0002870296C6520616E696D0A007428652993
:1002E00073742C20286D296F64652C20642875296F
:1002F0006D700A00506C61792053286E29616B651E
:100300000A00416C6C204C454473204F66662F4FA9
:100310006E2028302F31290A002832293A205465CE
:10032000737420416E696D2E20310A002833293AFA
:1003300020466F6E7420546573740A005379737489
:10034000656D2054696D653A2000204672616D65C7
:10035000732073746F7265640A004E657720616E56
:10036000696D6174696F6E20636F756E743A2000F9
:10037000647572617469286F296E0A004672616D36
:100380006520746F206368616E67653A200053656D
:100390006C662D546573743A203062004B696C6C46
:1003A000656420416E696D6174696F6E20436F757D
:1003B0006E746572210A00436F756C64206E6F74F1
:1003C0002061636365737320646576696365210AE0
:1003D00000417564696F20446174613A0A00436F9B
:1003E0006E74726F6C733A20572041205320442062
:1003F0005120452C207820746F20717569740A0093
:1004000052616E206F7574206F662048656170219F
:100410000A00416E696D6174696F6E2061626F726E
:10042000746564210A002869296E7465727275709A
:100430007420636F756E742C20287229616E646F4E
:100440006D2C2028712972657365740A0020496E2D
:100450007465727275707473206166746572203190
:100460003030306D7365630A00204672616D6573CC
:1004700020706572205365636F6E640A004D656D70
:100480006F72792064656C65746564210A00526539
:1004900073657420696E203530306D732E2042797B
:1004A00065210A00456E746572206672616D652073
:1004B000746F2064756D703A2000466F726D6174C0
:1004C00074696E67206D656D6F72792E2E2E200017
:1004D000446F6E65210A002866296F726D61742071
:1004E0006D656D6F72792C2028772972697465208B
:1004F000746578740A004475726174696F6E3A208D
:100500000053746172743A200038204C617965722E
:1005100062797465732E2E2E0A0053746F72696EA1
:100520006720696E2038206672616D65732E2E2EED
:100530000A00456E64653A200043756265206D6F60
:10054000646520656E7465726564210A0041756496
:10055000696F206D6F646520656E746572656421D6
:100560000A00546578743A2000E801EE0102021096
:10057000022B02470263029202BD02DC02F4020275
:100580000319032C033C034A035A0370037C038EB4
:10059000039C03B703D103DE030004120426044DB9
:1005A0000469047D048E04A404BA04D004D704F6BC
:1005B00004010509051A05320539054D0562055383
:1005C0007472696E67206E6F7420666F756E642139
:1005D0000A0000000000000000000C1E1E0C0C00B1
:1005E0000C00363636000000000036367F367F3687
:1005F00036000C3E031E301F0C00006333180C66DF
:1006000063001C361C6E3B336E00060603000000C0
:100610000000180C0606060C1800060C1818180C1A
:10062000060000663CFF3C660000000C0C3F0C0C12
:10063000000000000000000E0C060000003F00005B
:10064000000000000000000C0C006030180C0603D5
:1006500001001E333B3F37331E000C0F0C0C0C0CFB
:100660003F001E33301C06333F001E33301C303336
:100670001E00383C36337F3030003F031F303033AC
:100680001E001C06031F33331E003F3330180C06B8
:1006900006001E33331E33331E001E33333E301824
:1006A0000E0000000C0C000C0C0000000C0C000EE6
:1006B0000C06180C0603060C180000003F003F0053
:1006C0000000060C1830180C06001E3330180C0001
:1006D0000C003E637B7B7B031E000C1E33333F33D9
:1006E00033003F66663E66663F003C660303036672
:1006F0003C003F36666666363F007F46161E16464D
:100700007F007F46161E16060F003C6603037366C5
:100710007C003333333F333333001E0C0C0C0C0C92
:100720001E007830303033331E006766361E366662
:1007300067000F06060646667F0063777F6B63637C
:10074000630063676F7B736363001C3663636336A8
:100750001C003F66663E06060F001E3333333B1E09
:1007600038003F66663E1E3667001E33071C38336E
:100770001E003F2D0C0C0C0C1E003333333333336F
:100780003F0033333333331E0C006363636B7F7777
:1007900063006363361C366363003333331E0C0C13
:1007A0001E007F33190C46637F001E0606060606F0
:1007B0001E0003060C18306040001E181818181888
:1007C0001E00081C3663000000000000000000004E
:1007D00000FF0C0C18000000000000001E303E332B
:1007E0006E0007063E6666663D0000001E3303335A
:1007F0001E003830303E33336E0000001E333F039E
:100800001E001C36060F06060F0000006E33333E36
:10081000301F0706366E666667000C000E0C0C0C67
:100820001E0018001E1818181B0E070666361E3606
:1008300067000E0C0C0C0C0C1E000000377F6B6365
:10084000630000001F333333330000001E333333A3
:100850001E0000003B66663E060F00006E33333E0E
:10086000307800001B3636060F0000003E031E30B5
:100870001F00080C3E0C0C2C1800000033333333DF
:100880006E0000003333331E0C00000063636B7F87
:100890003600000063361C36630000003333333EFD
:1008A000301F00003F190C263F00380C0C070C0CC1
:1008B00038001818180018181800070C0C380C0C01
:1008C00007006E3B00000000000011241FBECFE5B2
:1008D000D8E0DEBFCDBF11E0A0E6B0E0EEECF8E579
:1008E00002C005900D92AA3DB107D9F712E0AAED1A
:1008F000B1E001C01D92A13EB107E1F70E940307DC
:100900000C94652C0C9400008FEF8ABB8CEF81BB9C
:1009100098E197BB84BB87B3866087BBB8980E9479
:10092000760A89E190E068E040E021E00E946D08ED
:100930000E94BB0A0E943E0C789485E690E00E94DB
:10094000150A0895CF93DF930E94200CC1E0009711
:1009500009F0C0E060E070E0CB0141E00E94590B7B
:10096000009711F4C26002C00E94D82980E063E2BF
:100970000E943C0D80E00E944A0D833211F0C46059
:1009800002C0CC2341F181E00E94590D0E9443092D
:10099000DC2F8C2F90E062E872E042E050E00E9491
:1009A000E22B0E9443098AE00E940309C0FF05C0B0
:1009B00083E00E94590D0E944309D1FF05C084E0E5
:1009C0000E94590D0E944309D2FF05C085E00E9494
:1009D000590D0E9443098C2FDF91CF910895AF925A
:1009E000BF92CF92DF92EF92FF920F931F93CF931C
:1009F000DF9380E490E00E943E29C82FD92F2097F2
:100A000031F488E10E94590D0E9443094EC0E82F3D
:100A1000F92FCF01805C9F4F1192E817F907E1F79A
:100A200000E010E191E0C92ED12CA895CE010E94E2
:100A3000150A0E94720A8823E1F30E94B52A5C011C
:100A40000E94B52A7C010E94B52A9C01C701B80109
:100A50000E94B328E62FF0E083E0EE0FFF1F8A9597
:100A6000E1F7C501B8010E94B328E60FF11DEC0FB4
:100A7000FD1FC901B8010E94B328C60102C0880F3A
:100A8000991F6A95E2F7BC018081862780830E94C6
:100A90009F08882351F289E10E94590D0E94430961
:100AA000CE010E94D8290E94AD08DF91CF911F91FD
:100AB0000F91FF90EF90DF90CF90BF90AF9008958F
:100AC000CF92DF92EF92FF920F931F93CF93DF931A
:100AD00090E0C0978A34910508F089C1865D9F4FE8
:100AE000FC01EE0FFF1F0590F491E02D099482E4C4
:100AF0007FC186E00E94590D0E94430987E00E9451
:100B0000590D0E94430988E00E94590D0E94430933
:100B100089E00E94590D0E9443098AE00E94590D04
:100B20000E9443098AE10E94590D0E94430982E212
:100B30000E94590D0E94430981E10E94590D0E94B3
:100B400043098BE00E94590D0E9443098CE00E94EA
:100B5000590D0E9443098DE012C180E090E00E948F
:100B60002B0D82E40E9403090CC080E20E94590D03
:100B70000E9443090E94EF0C81E20E94590D0E94DD
:100B8000430981E08093DB0135C10E94421932C1E3
:100B90000E94F313F6CF80E0F2C08091DC0188233D
:100BA00011F48091A50081508093DC018091DC01DB
:100BB000882341F06AE00E94D01A80E20E94030973
:100BC00089E2DDC088E2DBC081E08093DA018EE15A
:100BD000D6C00E94EF040EC10E9477190BC10E947B
:100BE000461908C10E940F0D62E872E04AE050E029
:100BF0000E94E22B0E94430980E690E00E94430994
:100C00008091DB0190E062E872E04AE050E00E94EF
:100C1000E22B0E94430983E690E00E9443098FE0A3
:100C2000AEC08FE10E94590D0E9443098AE00E94E4
:100C3000BD1A90E00E94BD0CEC010E94311A4EC01A
:100C400084E20E94590D0E9443098AE00E94BD1A65
:100C5000C82F87E20E94590D0E9443098AE00E9432
:100C6000BD1AE82E83E20E94590D0E9443098AE0D2
:100C70000E94BD1A082F06C08C2F90E0602F0E94A2
:100C8000DE0CCF5FEC16C0F781E279C08AE20E94E9
:100C9000590D0E9443090E94751BACC080E10E945F
:100CA000590D0E9443098AE00E94BD1A90E00E94FB
:100CB0002B0D67CF0E94221B9DC082E10E94590D1F
:100CC0000E9443098AE00E94BD1A082F0E94E01A80
:100CD000EC01802F90E0BE010E94CD0CCE010E945D
:100CE000D82988C00E94A20485C080E001C08FEF8F
:100CF0000E944A0A81E08093DF017CC085E690E093
:100D00000E94700DDD2441E0E42EF12C29C01882F0
:100D100000E010E0C701002E02C0880F991F0A945E
:100D2000E2F72881282B288385E690E00E94150AA7
:100D300005C0A8950E949F088823F1F40E94720ABA
:100D40008823B9F30F5F1F4F0830110519F7CA94B4
:100D50002196CC20E1F6D394FD2DF83008F0DD2467
:100D6000CD2DD0E033E0CC0FDD1F3A95E1F7CB5924
:100D7000DF4F28E0C22ECBCF0E94AD0889E10E9450
:100D8000590D0E94430936C085E690E00E94700D1F
:100D9000C0E08C2F0E941E1CCF3F11F0CF5F01C01E
:100DA000C0E0282F392FD901E5E6F0E08D9181933D
:100DB00080E0ED36F807D1F7CF0108970E94150AB9
:100DC00005C0A8950E949F088823B1F60E94720A68
:100DD0008C30F8F6F6CF0E940A0A42E852E02AE088
:100DE00030E00E94032C0E9443098AE001C083E2A4
:100DF0000E940309DF91CF911F910F91FF90EF9017
:100E0000DF90CF900895BF92CF92DF92EF92FF9242
:100E10000F931F93CF93DF9314BE88E10FB6F8941E
:100E200081BD11BC0FBE0E9484042EE088E190E0D9
:100E30000FB6F894A89581BD0FBE21BD0E94A204F3
:100E400090E080FF03C021E02093DD018670907068
:100E5000009719F081E08093DE0180E00E94590D37
:100E60000E9443098091DE01882321F40E940F0D26
:100E7000D82E01C0DD240E945D12C82F8091DD01B3
:100E8000882329F40E94D60D8F5F8093A50081E00E
:100E90008093DC0182E00E94590D0E944309BB242B
:100EA000EE24FF24CC24C394D0E021978091DA0172
:100EB000882309F4A8958091DB01882349F01092DA
:100EC000DB018091DE01882319F40E940F0DD82EDA
:100ED0000E949F08882321F00E94AD080E946005AF
:100EE0008091E001882371F080E0B09B21C0E7E8A9
:100EF000F1E03197F1F700C000008150B1F7109296
:100F0000E00116C080E0B09913C0E7E8F1E0319746
:100F1000F1F700C000008150B1F7C092E00180916C
:100F2000DC01882311F48091A50081508093DC01BD
:100F30008091DC01882309F03FC08091DF01882384
:100F400009F0B4CFDD2031F18091DE01882311F565
:100F50000E94720AB81608F0A9CF8F2D90E02D2DAF
:100F600030E0215030408217930714F4F39401C00D
:100F7000FF248F2D90E00E94BD0C8C01009789F119
:100F8000FC01E05CFF4FB0800E94150AC8010E947E
:100F9000D8298CCF0E94720AB81608F087CF2E2D60
:100FA00030E02C173D0714F4E39401C0EE248E2D9D
:100FB0000E94DB13B82E7ACF8091DD018823C1F423
:100FC0000E94720A882309F471CF0E94200C0097B6
:100FD00031F06091DC0161500E94270E67CF1092C2
:100FE000DC0185E690E00E94150A58E1B52E5ECF3F
:100FF0001092DC015BCF1F920F920FB60F9211245B
:101000008F939F93EF93FF93E091E301F091E401BD
:101010008CB1E550FE4F80838091E3019091E40113
:101020008F31910550F48091E3019091E401019694
:101030009093E4018093E30104C01092E4011092C4
:10104000E301FF91EF919F918F910F900FBE0F9051
:101050001F9018951F920F920FB60F9211242F9385
:101060003F938F939F93EF93FF932091E5013091EE
:10107000E6018091E7019091E80128173907F1F026
:10108000E091E501F091E601E55EFD4F80818CB9CC
:101090008091E5019091E6018F31910550F48091A6
:1010A000E5019091E60101969093E6018093E501B8
:1010B00009C01092E6011092E50104C081E080931E
:1010C000A6005598FF91EF919F918F913F912F919D
:1010D0000F900FBE0F901F901895433060F5362F7C
:1010E0003550343040F5322F3150323030F5442312
:1010F00041F030B5306230BD423019F430B5306166
:1011000030BD223019F420B5286020BD653061F073
:10111000663011F0683029F420B5226020BD6630B9
:1011200019F020B5246020BD90BD89B98AB18869C5
:101130008AB980E0089581E0089581E008954091A2
:10114000E1015091E2012091E3013091E40181E05D
:101150004217530709F480E008952091E10130918E
:10116000E2018091E3019091E4012817390729F108
:10117000E091E101F091E201E550FE4F8081E091C4
:10118000E101F091E201E550FE4F10822091E10172
:101190003091E2012F31310558F42091E101309175
:1011A000E2012F5F3F4F3093E2012093E101089568
:1011B0001092E2011092E101089580E0089580917B
:1011C000E7019091E8012091E5013091E601019657
:1011D0008217930791F08091E5019091E6010097C5
:1011E00079F42091E7013091E80181E090E02F311E
:1011F000310541F080E090E0089581E090E00895AD
:1012000080E090E008952091E7013091E80140915D
:10121000E5015091E6012F5F3F4F2417350799F301
:101220002091E5013091E6012115310539F4209135
:10123000E7013091E8012F31310529F3E091E70111
:10124000F091E801E55EFD4F80838091E701909188
:10125000E8018F31910550F48091E7019091E80108
:1012600001969093E8018093E70104C01092E80191
:101270001092E7018091A600813021F41092A6001F
:10128000559A5D9A0895CF93DF93C82FD92F02C046
:101290000E94030989918823D9F7DF91CF9108959E
:1012A0001AB810BC10BC19B81092E2011092E101FA
:1012B0001092E6011092E5011092E4011092E30110
:1012C0001092E8011092E70108951F920F920FB655
:1012D0000F9211242F933F934F935F936F938F93AC
:1012E0009F93AF93BF93EF93FF938091EC01809115
:1012F000E901882321F01092EB011092E90112BA62
:1013000088B3877E88BB80E090E021E030E045B381
:10131000437045BB48B3497F48BBE091EB01F0E027
:1013200043E0EE0FFF1F4A95E1F7E80FF91FE55C78
:10133000FD4F40814BBB823058F065B3A901082EA8
:1013400002C0440F551F0A94E2F7642B65BB0CC022
:1013500068B3AC014F5F5F4FF90102C0EE0FFF1F92
:101360004A95E2F76E2B68BB01968830910579F6B5
:101370002091EB0181E090E0AC0102C0440F551FC9
:101380002A95E2F742BB28B33091EB0102C0880FE7
:10139000991F3A95E2F733E0880F991F3A95E1F7E4
:1013A0008871277E822B88BB8091EB01873030F4D7
:1013B0008091EB018F5F8093EB0107C01092EB01EE
:1013C0008091EA018F5F8093EA011092EC01809195
:1013D000ED019091EE01A091EF01B091F001019625
:1013E000A11DB11D8093ED019093EE01A093EF013B
:1013F000B093F001FF91EF91BF91AF919F918F91C9
:101400006F915F914F913F912F910F900FBE0F9071
:101410001F9018952091ED013091EE014091EF0160
:101420005091F001B901CA010895CF93DF936FB7CE
:10143000F89421E02093E9011092EA011092EC0166
:10144000482F592F87E090E01DC0ED91F0E0E85162
:10145000FF4FE491E095E90173E0CC0FDD1F7A9531
:10146000E1F7C80FD91FC55CDD4FE8832F5F3F4F01
:101470002830310551F7485F5F4F01972FEF8F3FBD
:10148000920721F0DA0120E030E0DFCF6FBFDF917B
:10149000CF9108959FB7F89421E02093E90110922D
:1014A000EA011092EC0120E030E0809510C0FB01D1
:1014B000E40FF51FE55CFD4F80834F5F5F4F4830C1
:1014C0005105A9F72F5F3F4F2830310549F040E023
:1014D00050E0B901E3E0660F771FEA95E1F7E7CF47
:1014E0009FBF08958091EA01869508958EB5896021
:1014F0008EBD82EC92EA9BBD8ABD80E189BF80E00F
:101500000E944A0A789480E090E061E01DC07FB7B5
:10151000F894FA01E20FF31FE55CFD4FA081108201
:101520006093E9011092EA011092EC017FBF709183
:10153000EA017723E1F32F5F3F4F2830310539F778
:1015400001968830910549F020E030E0AC01F3E0ED
:10155000440F551FFA95E1F7DACFF8941092ED0198
:101560001092EE011092EF011092F0011092EA0138
:101570001092EC01089511B88CE080B9089594EAB6
:1015800096BF06B607FEFDCF91B1987F983011F057
:10159000903179F483B984E886BF06B607FEFDCFA3
:1015A00091B1987F983139F081E0903429F480E04E
:1015B000089581E0089580E0089544EA34E824E93C
:1015C00046BF06B607FEFDCF91B1987F983011F067
:1015D0009031B1F783B936BF06B607FEFDCF91B1A2
:1015E000987F903211F0983529F426BF06B604FC96
:1015F000FDCFE6CF08950E94BF0A089584E986BF13
:1016000006B604FCFDCF089583B984E886BF06B60C
:1016100007FEFDCF91B1987F81E0983209F480E018
:10162000089584EC86BF06B607FEFDCF83B108950A
:1016300084E886BF06B607FEFDCF83B10895DF922A
:10164000EF92FF920F931F93DF93CF930F92CDB73B
:10165000DEB77B018C0180E0E81680E0F80681E0CF
:10166000080780E0180718F490EAD92E02C082EA31
:10167000D82E8D2D0E94BF0A882389F48F2D0E94B9
:10168000040B8E2D0E94040B8D2D81600E94FB0A9D
:101690000E94180B89830E94FE0A898101C080E0A4
:1016A0000F90CF91DF911F910F91FF90EF90DF90FE
:1016B00008958F929F92AF92BF92CF92DF92EF9256
:1016C000FF920F931F93CF93DF934B015C0180E058
:1016D000881680E0980681E0A80680E0B80618F435
:1016E00030EAE32E02C022EAE22E042F10E0C80105
:1016F0000E943E29EC016C01009731F488E10E94C0
:10170000590D0E9443092CC08E2D0E94BF0A8823C8
:1017100029F5892D0E94040B882D0E94040B8E2D23
:1017200081600E94FB0ABB2448010894810891084B
:1017300007C00E94110BFE01EE0DFF1D8083B394C4
:10174000EB2CFF24E814F904A4F30E94180BC00F3B
:10175000D11F219788830E94FE0A02C0CC24DD2479
:10176000C601DF91CF911F910F91FF90EF90DF9015
:10177000CF90BF90AF909F908F900895EF92FF927F
:101780000F931F93CF937B018C01C42F80E0E81649
:1017900080E0F80681E0080780E0180710F480EA8E
:1017A00001C082EA0E94BF0A882359F48F2D0E944B
:1017B000040B8E2D0E94040B8C2F0E94040B0E94A0
:1017C000FE0ACF911F910F91FF90EF900895CF9255
:1017D000DF92EF92FF920F931F93CF93DF937B01E2
:1017E0008C01D42EC52FC22E80E0E81680E0F806CA
:1017F00081E0080780E0180710F480EA01C082EA5F
:101800000E94BF0A882399F48F2D0E94040B8E2D0D
:101810000E94040B8C2FCD2DD82F03C089910E94DC
:10182000040B8C2F8D198C15C8F30E94FE0ADF91D2
:10183000CF911F910F91FF90EF90DF90CF9008957F
:10184000CF93DF9383E40E94BF0A882389F4CBE718
:10185000D2E00E94110B899382E0C138D807C9F702
:101860000E94180B809381020E94FE0A269702C0F4
:10187000C0E0D0E0CE01DF91CF91089583B78B60B7
:1018800083BF8AEF8CBF89B7826089BF08951F929A
:101890000F920FB60F9211242F933F934F935F93A4
:1018A0006F937F938F939F93AF93EF93FF934091A9
:1018B000F2013091F3012091F4019091F5018091B2
:1018C000F601F091F701E091F801A091F901642F80
:1018D0006F5F51E0641708F050E0530F41E0531779
:1018E00008F040E0420F31E0421708F030E0390FD5
:1018F00021E0391708F020E0280F91E0281708F0C0
:1019000090E09F0F81E09F1708F080E08E0F71E05C
:101910008E1708F070E07A0F6093F2015093F30194
:101920004093F4013093F5012093F6019093F70171
:101930008093F8017093F901FF91EF91AF919F911E
:101940008F917F916F915F914F913F912F910F9068
:101950000FBE0F901F9018952091F2013091F30166
:101960004091F4015091F5016091F6017091F701F9
:101970008091F8019091F9010895BC0126E0660F6D
:10198000771F2A95E1F7680F791F605E7F4F80E02F
:1019900090E041E40E94590B0895AB01BC0136E090
:1019A000660F771F3A95E1F7680F791F605E7F4FEA
:1019B00080E090E021E40E94E70B0895462F9C010F
:1019C00056E0220F331F5A95E1F7280F391F205A8E
:1019D0003F4FB90180E090E00E94BE0B0895EF9266
:1019E000FF920F931F93EE24FF248701C801B701D4
:1019F00040E00E94BE0BA8950894E11CF11C011D5B
:101A0000111D80E0E81680E0F80682E0080780E01B
:101A1000180761F71F910F91FF90EF900895CF93F2
:101A200060E070E0CB010E941F0BC82F61E070E006
:101A300080E090E00E941F0B2C2F30E0582F40E0F8
:101A4000242B352B87E0213E380710F020EE37E0BD
:101A5000C901CF910895CF93482FC92F60E070E05E
:101A6000CB010E94BE0B61E070E080E090E04C2F63
:101A70000E94BE0BCF910895462F8E3150F490E016
:101A800002969C01B901882777FD8095982F0E94C6
:101A9000BE0B08958E3158F4682F70E06E5F7F4F53
:101AA000882777FD8095982F0E941F0B089580E06E
:101AB00008958B3248F4E82FF0E0EE0FFF1FE7594E
:101AC000FA4F2591349104C0EFEBF5E02591349164
:101AD00082E892E0B9010E94DB2B82E892E008954F
:101AE000282F392FF90180E411928150E9F70895E8
:101AF0001F93CF93DF9381E490E00E943E29192F3A
:101B0000C82FD92F209731F488E10E94590D0E94E7
:101B10004309FFCFCE010E94700DFE01E05CFF4F34
:101B200081E080838C2F912FDF91CF911F910895B9
:101B3000A7E0B0E0FD01E41BF109AD01421B510932
:101B40009A0143E0220F331F4A95E1F7E20FF31F9A
:101B5000E80FF91F81E090E002C0880F991F6A9595
:101B6000E2F72081282B20830895A7E0B0E0FD0153
:101B7000E41BF109AD01421B51099A0153E0220F08
:101B8000331F5A95E1F7E20FF31FE80FF91F81E0C9
:101B900090E002C0880F991F6A95E2F780959081C6
:101BA0009823908308950E94D829089587E0089586
:101BB000282F392FF90197E080E02191821708F44E
:101BC000822F9150D1F70895982F662359F0E5EBB5
:101BD000F0E080E003C08F5F883039F02191291751
:101BE000D0F308956FE10E9493280895282F392F8C
:101BF000F90127E080E090E03191830F911D2150A1
:101C0000D9F767E070E00E949F28862F08951F9300
:101C1000CF93DF93D82FC92F662321F00E94F60DB2
:101C2000823110F412E101C019E08D2F9C2F0E9427
:101C3000F60D811740F49E01832F922FFC0187E05F
:101C400011928150E9F7DF91CF911F9108951F9371
:101C5000CF93DF93EC01162F6730C0F4662321F099
:101C6000862F8450823018F4CE0161E002C0CE018C
:101C700060E00E94070EE12FF0E0EE0FFF1FE95534
:101C8000FF4F0190F081E02DCE010995DF91CF91BA
:101C90001F9108956F927F928F929F92AF92BF9201
:101CA000CF92DF92EF92FF920F931F93CF93DF9328
:101CB0007B01142F622EC02EA82EB92E01E09FE0CA
:101CC000892E912CF50181915F01662D0E94E40D12
:101CD000782EC0E0D0E0DD2429C00130C1F4CC2052
:101CE00059F0CE01B4010E94B328262FC70160E04D
:101CF000412F0E94980D0DC0CE01B4010E94B3285F
:101D0000462FC70160E0212F0E94980D07C0CC200C
:101D100029F0C701602F412F2D2D04C0C701602F6E
:101D20004D2D212F0E94980DD3942A96D714A8F2F6
:101D30000F5F083039F6DF91CF911F910F91FF901F
:101D4000EF90DF90CF90BF90AF909F908F907F905B
:101D50006F900895EF92FF920F931F93CF93DF93AD
:101D60007C010E94780DEC0110E0C701BE01412FFB
:101D700020E000E00E944A0E1F5F1830B1F7CE014C
:101D80000E94150ACE010E94D30DDF91CF911F91C1
:101D90000F91FF90EF900895EF92FF920F931F9392
:101DA000CF93DF937C010E94780DEC0110E0C70116
:101DB000BE01412F21E000E00E944A0E1F5F183053
:101DC000B1F7CE010E94150ACE010E94D30DDF911A
:101DD000CF911F910F91FF90EF900895EF92FF9296
:101DE0000F93CF93DF937C010E94780DEC01C70124
:101DF000BE0142E021E000E00E944A0EC70160E01F
:101E00000E94070EC701BE0145E020E00E944A0E75
:101E1000CE010E94150ACE010E94D30DDF91CF9111
:101E20000F91FF90EF900895EF92FF920F931F9301
:101E3000CF93DF937C010E94780DEC0112E0C70183
:101E4000BE01412F20E001E00E944A0E1F5F1630C4
:101E5000B1F7CE010E94150ACE010E94D30DDF9189
:101E6000CF911F910F91FF90EF9008950F931F93C3
:101E7000CF93DF938C010E94780DEC01C801BE0165
:101E800047E020E000E00E944A0ECE010E94150AC1
:101E9000CE010E94D30DDF91CF911F910F91089534
:101EA0000F931F93CF93DF938C010E94780DEC0169
:101EB000C801BE0147E021E000E00E944A0ECE01C9
:101EC0000E94150ACE010E94D30DDF91CF911F9180
:101ED0000F910895EF92FF920F931F93CF93DF938B
:101EE000F82E062F142FE901EE2407C0CE016F2D26
:101EF0004E2D202F0E94980DE394E116B8F3DF9148
:101F0000CF911F910F91FF90EF900895FF920F9343
:101F10001F93CF93DF938C010E94780DEC01F801A1
:101F200080812FE1F22E6F2D0E949328482F80E0B0
:101F300060E09E010E946A0FF80180816F2D0E946F
:101F40009328482F80E061E09E010E946A0FF8010B
:101F500080816F2D0E949328482F81E060E09E01D0
:101F60000E946A0FF80181816F2D0E949328482FEB
:101F700080E062E09E010E946A0FF80181816F2D6E
:101F80000E949328482F80E063E09E010E946A0F20
:101F9000F80181816F2D0E949328482F81E061E034
:101FA0009E010E946A0FF80181816F2D0E94932883
:101FB000482F81E062E09E010E946A0FF801818152
:101FC0006F2D0E949328482F82E060E09E010E94BE
:101FD0006A0FF80181816F2D0E949328482F82E0BB
:101FE00061E09E010E946A0FF80182816F2D0E94BC
:101FF0009328482F80E064E09E010E946A0FF80158
:1020000082816F2D0E949328482F80E065E09E0119
:102010000E946A0FF80182816F2D0E949328482F39
:1020200081E063E09E010E946A0FF80182816F2DBA
:102030000E949328482F81E064E09E010E946A0F6D
:10204000F80182816F2D0E949328482F82E062E080
:102050009E010E946A0FF80182816F2D0E949328D1
:10206000482F82E063E09E010E946A0FF80182819E
:102070006F2D0E949328482F83E060E09E010E940C
:102080006A0FF80182816F2D0E949328482F83E008
:1020900061E09E010E946A0FF80182816F2D0E940B
:1020A0009328482F83E062E09E010E946A0FF801A6
:1020B00082816F2D0E949328482F84E060E09E016A
:1020C0000E946A0FF80182816F2D0E949328482F89
:1020D00084E061E09E010E946A0FF80183816F2D08
:1020E0000E949328482F80E066E09E010E946A0FBC
:1020F000F80183816F2D0E949328482F80E067E0CC
:102100009E010E946A0FF80183816F2D0E9493281F
:10211000482F81E065E09E010E946A0FF8018381EB
:102120006F2D0E949328482F81E066E09E010E9457
:102130006A0FF80183816F2D0E949328482F82E057
:1021400064E09E010E946A0FF80183816F2D0E9456
:102150009328482F82E065E09E010E946A0FF801F3
:1021600083816F2D0E949328482F83E063E09E01B6
:102170000E946A0FF80183816F2D0E949328482FD7
:1021800083E064E09E010E946A0FF80183816F2D55
:102190000E949328482F84E062E09E010E946A0F0B
:1021A000F80183816F2D0E949328482F84E063E01B
:1021B0009E010E946A0FF80183816F2D0E9493286F
:1021C000482F85E060E09E010E946A0FF80183813C
:1021D0006F2D0E949328482F85E061E09E010E94A8
:1021E0006A0FF80183816F2D0E949328482F85E0A4
:1021F00062E09E010E946A0FF80183816F2D0E94A8
:102200009328482F86E060E09E010E946A0FF80143
:1022100083816F2D0E949328482F86E061E09E0104
:102220000E946A0FF80184816F2D0E949328482F25
:1022300081E067E09E010E946A0FF80184816F2DA2
:102240000E949328482F82E066E09E010E946A0F58
:10225000F80184816F2D0E949328482F82E067E067
:102260009E010E946A0FF80184816F2D0E949328BD
:10227000482F83E065E09E010E946A0FF801848187
:102280006F2D0E949328482F83E066E09E010E94F4
:102290006A0FF80184816F2D0E949328482F84E0F3
:1022A00064E09E010E946A0FF80184816F2D0E94F4
:1022B0009328482F84E065E09E010E946A0FF80190
:1022C00084816F2D0E949328482F85E063E09E0152
:1022D0000E946A0FF80184816F2D0E949328482F75
:1022E00085E064E09E010E946A0FF80184816F2DF1
:1022F0000E949328482F86E062E09E010E946A0FA8
:10230000F80184816F2D0E949328482F86E063E0B6
:102310009E010E946A0FF80184816F2D0E9493280C
:10232000482F87E060E09E010E946A0FF8018481D7
:102330006F2D0E949328482F87E061E09E010E9444
:102340006A0FF80185816F2D0E949328482F83E042
:1023500067E09E010E946A0FF80185816F2D0E943F
:102360009328482F84E066E09E010E946A0FF801DE
:1023700085816F2D0E949328482F84E067E09E019D
:102380000E946A0FF80185816F2D0E949328482FC3
:1023900085E065E09E010E946A0FF80185816F2D3E
:1023A0000E949328482F85E066E09E010E946A0FF4
:1023B000F80185816F2D0E949328482F86E064E004
:1023C0009E010E946A0FF80185816F2D0E9493285B
:1023D000482F86E065E09E010E946A0FF801858122
:1023E0006F2D0E949328482F87E062E09E010E9493
:1023F0006A0FF80185816F2D0E949328482F87E08E
:1024000063E09E010E946A0FF80185816F2D0E9492
:102410009328482F87E064E09E010E946A0FF8012C
:1024200086816F2D0E949328482F85E067E09E01EA
:102430000E946A0FF80186816F2D0E949328482F11
:1024400086E066E09E010E946A0FF80186816F2D8A
:102450000E949328482F86E067E09E010E946A0F41
:10246000F80186816F2D0E949328482F87E065E050
:102470009E010E946A0FF80186816F2D0E949328A9
:10248000482F87E066E09E010E946A0FF80186816E
:102490006F2D0E949328482F87E067E09E010E94DD
:1024A0006A0FCE010E94150ACE010E94D30DDF9162
:1024B000CF911F910F91FF90089580E108958F9221
:1024C0009F92AF92BF92CF92DF92EF92FF920F93C3
:1024D0001F93DF93CF9300D0CDB7DEB7882E0E9435
:1024E000780D7C01B82CBB0C99240894811C911C9C
:1024F000880C991C00E010E0CB2CDD24C7FCD094A4
:1025000024C0C701632F4A2D252F3A8359830E9487
:10251000980D59815F5F3A81583099F73F5F3830A5
:1025200021F405C030E0AB2CA00E50E0EACFC7018B
:102530000E94150A01C0A8950E94720A8823D9F347
:10254000C7010E94700D0F5F1F4FC8018C0D9D1DAC
:10255000881599053CF3C7010E94D8290F900F9068
:10256000CF91DF911F910F91FF90EF90DF90CF906F
:10257000BF90AF909F908F9008958F929F92BF923F
:10258000CF92DF92EF92FF920F931F93DF93CF933F
:1025900000D0CDB7DEB7E82E0E94780D8C01BE2C9E
:1025A000B194BB0C23E0822E912C8E189108880CDC
:1025B000991C87E0B80EEE24FF24CB2CDD24C7FC49
:1025C000D09424C0C801632F4B2D252F3A83598303
:1025D0000E94980D59815F5F3A81583099F73F5FAB
:1025E000383011F403C030E050E0ECCFC8010E9455
:1025F000150A01C0A8950E94720A8823D9F3C80160
:102600000E94700DBA940894E11CF11CC6018E1949
:102610009F09881599053CF7C8010E94D8290F9099
:102620000F90CF91DF911F910F91FF90EF90DF906E
:10263000CF90BF909F908F9008958F929F92AF926E
:10264000BF92CF92DF92EF92FF920F931F93DF938F
:10265000CF9300D0CDB7DEB7882E0E94780D7C01D5
:10266000B82CBB0C99240894811C911C880C991CD3
:1026700000E010E0CB2CDD24C7FCD09424C0C701BF
:10268000652F432F2A2D3A8359830E94980D598133
:102690005F5F3A81583099F73F5F383021F405C0C9
:1026A00030E0AB2CA00E50E0EACFC7010E94150A23
:1026B00001C0A8950E94720A8823D9F3C7010E941D
:1026C000700D0F5F1F4FC8018C0D9D1D881599055A
:1026D0003CF3C7010E94D8290F900F90CF91DF9152
:1026E0001F910F91FF90EF90DF90CF90BF90AF9030
:1026F0009F908F9008958F929F92BF92CF92DF927A
:10270000EF92FF920F931F93DF93CF9300D0CDB73B
:10271000DEB7E82E0E94780D8C01BE2CB194BB0C64
:1027200053E0852E912C8E189108880C991C87E017
:10273000B80EEE24FF24CB2CDD24C7FCD09424C09B
:10274000C801632F452F2B2D3A8359830E94980D82
:1027500059815F5F3A81583099F73F5F383011F403
:1027600003C030E050E0ECCFC8010E94150A01C060
:10277000A8950E94720A8823D9F3C8010E94700D9F
:10278000BA940894E11CF11CC6018E199F098815A2
:1027900099053CF7C8010E94D8290F900F90CF915E
:1027A000DF911F910F91FF90EF90DF90CF90BF903E
:1027B0009F908F9008958031A0F4843018F40E9487
:1027C0001D130FC0883020F484500E947B1309C071
:1027D0008C3020F488500E945F1203C08C500E94FD
:1027E000BD1281E008952F923F924F925F926F92B7
:1027F0007F928F929F92AF92BF92CF92DF92EF9291
:10280000FF920F931F93DF93CF93CDB7DEB76C97F3
:102810000FB6F894DEBF0FBECDBF81E490E00E94FA
:102820003E29888B998B8B839C830E94AC0CB22EA3
:10283000C32ED42E152F062FF72EE82E392E82E424
:102840000E94030974C00E94AC0CA22FAB19F1E0E6
:102850002A1708F0F0E0232F2C19E1E0321708F0D6
:10286000E0E0322F3F1BF32F31E02F1708F030E06C
:10287000E32B342F3D1921E0431708F020E0432FCC
:102880004E1BE42F41E03E1708F040E0242B452F7B
:10289000411B31E0541708F030E0542F521B21E067
:1028A000451708F020E0322B462F401B21E064172B
:1028B00008F020E0642F631B31E0461708F030E099
:1028C000232B472F4F1931E0741708F030E0742F95
:1028D000721B21E0471708F020E0322B482F4E19D9
:1028E00021E0841708F020E0842F831B31E0481793
:1028F00008F030E0232B9319921709F099C488232C
:1029000009F096C4772309F093C4662309F090C4B4
:10291000552309F08DC4EE2309F08AC4F23008F083
:1029200087C4F13019F4A53F08F082C4A8950E942D
:102930009F08882309F487CF0E94AD088A8B82E420
:102940000E94030984EF282EAA24A3945524662408
:1029500077248824992444241F821E821E868B811A
:102960009C81805C9F4F9F8B8E8B2D82BB86CC86FB
:10297000DD86212EB02ECF2CDE2C37C20E94AC0C6F
:10298000122FAB851A1BF1E0211708F0F0E0E32FBE
:10299000BC85EB1B21E03E1708F020E03E2F3F1BDB
:1029A000F1E0E31708F0F0E02F2BA42FED85AE1B2C
:1029B000F1E04A1708F0F0E04A2F421B21E0A4178B
:1029C00008F020E0F22BA52FA21921E05A1708F0F9
:1029D00020E05A2F5F1BF1E0A51708F0F0E02F2B45
:1029E000A62FAB19F1E06A1708F0F0E06A2F621B1E
:1029F00021E0A61708F020E0F22B272F2C19A1E0E8
:102A0000721708F0A0E0722F7F1BF1E0271708F083
:102A1000F0E0AF2BF82FFD1921E08F1708F020E030
:102A20008F2F8A1BA1E0F81708F0A0E02A2B93193A
:102A3000921B491608F4FCC3941511F5981608F476
:102A4000F7C38915E9F4871608F4F2C37815C1F4C1
:102A5000761608F4EDC3671599F4651608F4E8C313
:102A6000561571F4541608F4E3C3451549F4A3163A
:102A700008F4DEC33A1521F4FD81F11708F4D8C338
:102A8000A8950E949F08882309F478CF0E94AD087A
:102A90008B8B82E40E9403092E813F813A83298334
:102AA0004F864B2CBC2CCD2C8EC13D813C503A879F
:102AB00051E04D81341708F050E08A2D8F5F91E08E
:102AC0008A1508F090E0580F41E0581708F040E0F0
:102AD000492B450D11E0451508F010E0160D01E0F9
:102AE000161508F000E0070D81E0071508F080E0FA
:102AF000F82EF80C81E0F81408F080E0E82EE90CDC
:102B000081E0E91408F080E0DF84D80E8A858D83A7
:102B1000A52E542E612E702E8F2C9E2CDF86588F62
:102B20004C8B87C00E94AC0CA22FBB85AB1BA88727
:102B3000F1E02A1708F0F0E0E32F2C85E21B21E0FA
:102B40003E1708F020E03E2F3F1BF1E0E31708F0AE
:102B5000F0E02F2BA42FBD85AB1BF1E04A1708F046
:102B6000F0E04A2F421B21E0A41708F020E0F22BEE
:102B7000A52FA21921E05A1708F020E05A2F5F1B59
:102B8000F1E0A51708F0F0E02F2BA62FA419F1E033
:102B90006A1708F0F0E06A2F621B21E0A61708F020
:102BA00020E0F22B272F2B19A1E0721708F0A0E0EC
:102BB000722F7F1BF1E0271708F0F0E0AF2BF82F02
:102BC000FC1921E08F1708F020E08F2F8A1BA1E06D
:102BD000F81708F0A0E02A2B9319921BD91608F4D5
:102BE00027C39D1529F5E81608F422C38E1501F5B3
:102BF000F71608F41DC37F15D9F4061708F418C397
:102C00006017B1F4151708F413C3511789F4EC8950
:102C1000E41708F40DC34E1759F4F88DF31708F4B0
:102C200007C33F1729F428853A85321708F400C3F3
:102C3000A8950E949F08882309F474CF588D4C8969
:102C40004C8F5A8F0E94AD08AE89BF898C9382E465
:102C50000E94030938892989832F922F99878887B1
:102C6000805C9F4F9D8B8C8B5A8D5B8F4C8D498FD9
:102C70008AC00E94AC0CE22FBB85EB1BF1E02E1743
:102C800008F0F0E0232FAC852A1BB1E0B88F321793
:102C900008F0188E322F3F1BF32F31E02F1708F06A
:102CA00030E0A88DA32BA88F342FBD853B1B21E0DE
:102CB000431708F020E0432FA88D4A1BA1E03417EA
:102CC00008F0A0E02A2BA52FA21931E05A1708F02E
:102CD00030E05A2F521B21E0A51708F020E0322BDC
:102CE000A62FA41921E06A1708F020E06A2F631BC1
:102CF00031E0A61708F030E0232BA72FAB1931E005
:102D00007A1708F030E07A2F721B21E0A71708F03D
:102D100020E0322BA82FAC1921E08A1708F020E020
:102D20008A2F831B31E0A81708F030E0232B93197A
:102D3000921BD91608F47CC29D1521F5E81608F4FB
:102D400077C28E15F9F4F71608F472C27F15D1F424
:102D5000061708F46DC26017A9F4151708F468C2C5
:102D6000511781F4B98DB41708F462C24B1751F4AE
:102D70002B8D2F1708F45CC2F21721F43A853E1709
:102D800008F456C2A8950E949F08882309F471CFC1
:102D90000E94AD08A885B9858D93B987A887EC896D
:102DA000FD89AE17BF0779F782E40E940309098104
:102DB0001A810F5F1F4F89819A816B817C810E94EC
:102DC000CD0C1A8309838981FE818F1B2B89821781
:102DD00008F46BCEDC2CCB2CB42C4F843E853F5FAB
:102DE0003E8789819A819F838E839E85AA899A17BF
:102DF00008F447CE122D2D800B2DBB84FC2CCC84E7
:102E0000ED2CDD848B819C810E94D82980C00E949A
:102E1000AC0CE22FEB19F1E02E1708F0F0E0232FB5
:102E20002C19A1E0321708F0A0E0B22FBF1BFB2F36
:102E300031E02B1708F030E0A32B342F3D1921E0AF
:102E4000431708F020E0432F4A1BA1E0341708F095
:102E5000A0E02A2BA52FA11B31E05A1708F030E083
:102E60005A2F521B21E0A51708F020E0322BA62F85
:102E7000A01B21E06A1708F020E06A2F631B31E0F5
:102E8000A61708F030E0232BA72FAF1931E07A17EF
:102E900008F030E07A2F721B21E0A71708F020E03D
:102EA000322BA82FAE1921E08A1708F020E08A2FD4
:102EB000831B31E0A81708F030E0232B9319921BF5
:102EC000491608F4B5C1941509F5981608F4B0C16F
:102ED0008915E1F4871608F4ABC17815B9F47616B4
:102EE00008F4A6C1671591F4651608F4A1C156153A
:102EF00069F4541608F49CC1451541F4AF1608F462
:102F000097C1FA1519F42E1608F492C1A8950E94DB
:102F10009F08882309F47BCF0E94AD0880C00E94DF
:102F2000AC0CE22FEB19F1E02E1708F0F0E0232FA4
:102F30002C19A1E0321708F0A0E0322F3F1BF32F2D
:102F400031E02F1708F030E0A32B342F3D1921E09A
:102F5000431708F020E0432F4A1BA1E0341708F084
:102F6000A0E02A2BA52FA11B31E05A1708F030E072
:102F70005A2F521B21E0A51708F020E0322BA62F74
:102F8000A01B21E06A1708F020E06A2F631B31E0E4
:102F9000A61708F030E0232BA72FAF1931E07A17DE
:102FA00008F030E07A2F721B21E0A71708F020E02C
:102FB000322BA82FAE1921E08A1708F020E08A2FC3
:102FC000831B31E0A81708F030E0232B9319921BE4
:102FD000491608F42DC1941509F5981608F428C16E
:102FE0008915E1F4871608F423C17815B9F476162B
:102FF00008F41EC1671591F4651608F419C1561539
:1030000069F4541608F414C1451541F4AF1608F4D8
:103010000FC1FA1519F42E1608F40AC1A8950E94DA
:103020009F08882309F47BCF0E94AD0880C00E94CE
:10303000AC0CE22FEB19F1E02E1708F0F0E0232F93
:103040002C19A1E0321708F0A0E0B22FBF1BFB2F14
:1030500031E02B1708F030E0A32B342F3D1921E08D
:10306000431708F020E0432F4A1BA1E0341708F073
:10307000A0E02A2BA52FA11B31E05A1708F030E061
:103080005A2F521B21E0A51708F020E0322BA62F63
:10309000A01B21E06A1708F020E06A2F631B31E0D3
:1030A000A61708F030E0232BA72FAF1931E07A17CD
:1030B00008F030E07A2F721B21E0A71708F020E01B
:1030C000322BA82FAE1921E08A1708F020E08A2FB2
:1030D000831B31E0A81708F030E0232B9319921BD3
:1030E000491608F4A5C0941509F5981608F4A0C06F
:1030F0008915E1F4871608F49BC07815B9F47616A3
:1031000008F496C0671591F4651608F491C0561539
:1031100069F4541608F48CC0451541F4AF1608F450
:1031200087C0FA1519F42E1608F482C0A8950E94DB
:103130009F08882309F47BCF0E94AD087CC00E94C1
:10314000AC0CE22FEB19F1E02E1708F0F0E0232F82
:103150002C19A1E0321708F0A0E0322F3F1BF32F0B
:1031600031E02F1708F030E0A32B342F3D1921E078
:10317000431708F020E0432F4A1BA1E0341708F062
:10318000A0E02A2BA52FA11B31E05A1708F030E050
:103190005A2F521B21E0A51708F020E0322BA62F52
:1031A000A01B21E06A1708F020E06A2F631B31E0C2
:1031B000A61708F030E0232BA72FAF1931E07A17BC
:1031C00008F030E07A2F721B21E0A71708F020E00A
:1031D000322BA82FAE1921E08A1708F020E08A2FA1
:1031E000831B31E0A81708F030E0232B9319921BC2
:1031F0004916F0F09415D1F49816D0F08915B1F471
:103200008716B0F0781591F4761690F0671571F482
:10321000651670F0561551F4541650F0451531F4FA
:10322000AF1630F0FA1511F42E1610F0A89503C061
:1032300080E090E00CC00E949F08882309F47FCFB3
:103240000E94AD0882E40E9403098E819F810E9442
:103250002B0D6C960FB6F894DEBF0FBECDBFCF918D
:10326000DF911F910F91FF90EF90DF90CF90BF9073
:10327000AF909F908F907F906F905F904F903F9016
:103280002F90089583E20E94030908951F93CF931E
:10329000DF930E94200CEC01009731F485E10E943D
:1032A000590D0E9443091FC086E10E94590D0E94DA
:1032B000430910E3812F0E9403098DEB90E00E94E7
:1032C0004309899190E062E872E04AE050E00E9490
:1032D000E22B82E892E00E9443098AE00E940309FF
:1032E0001F5F173339F7DF91CF911F910895AF9288
:1032F000BF92CF92DF92EF92FF920F931F938EE0D7
:103300000E94590D0E9443090E94AC0CB901CA01E8
:1033100042E852E02AE030E00E94032C0E94430978
:1033200080EC90E00E9443090E94AC0C992381F448
:10333000882371F4772361F4662351F4552341F413
:10334000442331F43B3E20F43A3E09F52136F8F0AF
:1033500083EC90E00E9443090E94AC0CB0E6AB2ED7
:10336000AAEEBA2ECC24DD24EE24FF2400E010E0E7
:103370000E943F1CC90162E872E04AE050E00E94EE
:10338000E22B0E94430986EC90E00E9443090E94D0
:10339000AC0C992391F4882381F4772371F466238C
:1033A00061F4552351F4442341F4343030F4333084
:1033B00009F04BC0293E08F448C083EC90E00E941D
:1033C00043090E94AC0CF8EEAF2EE3E0BE2ECC24F5
:1033D000DD24EE24FF2400E010E00E943F1CC90120
:1033E00062E872E04AE050E00E94E22B0E9443094A
:1033F0000E94AC0C0E947322C90162E872E04AE0AC
:1034000050E00E94E22B80918202882319F08EE224
:103410000E94030980918402882319F480E30E94AA
:10342000030980918302882319F480E30E94030931
:1034300080918202882321F082E892E00E94430971
:103440008CEC90E00E94430903C08AE00E940309CB
:103450001F910F91FF90EF90DF90CF90BF90AF90B2
:103460000895AF92BF92DF92EF92FF920F931F9356
:10347000DF93CF930F92CDB7DEB77C015C0110E3F1
:10348000D12E8D2D0E9403098DEB90E00E944309FF
:10349000850120E0F80181918F0190E062E872E0FF
:1034A00040E150E029830E94E22B82E892E00E94F2
:1034B000430980E20E94030929812F5F283051F7D8
:1034C0008AE00E940309D39488E090E0A80EB91E18
:1034D0009D2D9833B1F683E20E94590D0E94430955
:1034E000F701E05CFF4F808190E062E872E04AE023
:1034F00050E00E94E22B82E892E00E9443098AE0B9
:103500000E9403090F90CF91DF911F910F91FF90BF
:10351000EF90DF90BF90AF900895FF920F931F93AD
:10352000CF93DF93FF24A8950E949F088823D9F3A7
:10353000CF2DD0E00E94AD088E010E571D4FF8012F
:1035400080830E940309F80180818A3019F0FF2DE1
:10355000F03559F4CE57DD4F188282E892E0DF91C2
:10356000CF911F910F91FF9008958D30E1F2883037
:1035700011F4FA94D8CFF394D6CFDF93CF930F9270
:10358000CDB7DEB789830E948D1A60E070E0498173
:1035900050E00E94C52A862F0F90CF91DF910895A9
:1035A000CF93DF93462FC2E8D2E090E0BE0150E017
:1035B0000E94E22BCE010E944309DF91CF91089532
:1035C000EF92FF920F931F93DF93CF930F92CDB79C
:1035D000DEB781E490E00E943E29182F092FE82EE3
:1035E000F92E83E20E94590D0E9443098AE00E944D
:1035F000BD1AF701E05CFF4F8083C801092F182F27
:1036000020E0822F6AE029830E94D01A8DEB90E09F
:103610000E94430980E10E94BD1AF80181938F0145
:1036200029812F5F203469F781E20E94590D0E94A1
:103630004309C7010F90CF91DF911F910F91FF9028
:10364000EF900895FF920F931F93DF93CF93CDB721
:10365000DEB729970FB6F894DEBF0FBECDBF8E013F
:103660000F5F1F4F88E0F80111928A95E9F784E215
:103670000E94590D0E9443098AE00E94BD1AF82E4B
:1036800085E20E94590D0E94430920E0822F6AE0E2
:1036900029870E94D01A8DEB90E00E94430980E1B7
:1036A0000E94BD1AF80181938F0129852F5F283070
:1036B00069F786E20E94590D0E944309CE010196E6
:1036C0006F2D42E00E949A1B81E20E94590D0E94D8
:1036D000430929960FB6F894DEBF0FBECDBFCF9138
:1036E000DF911F910F91FF900895CF93DF930E9478
:1036F0008D1AC2E8D2E0CE0160E00E94F91BFE0103
:1037000001900020E9F7CF0101978C1B9D0B23E06E
:10371000880F991F2A95E1F701960E942B0D81E0F1
:103720008093DB0181E20E94590D0E944309DF91E1
:10373000CF9108958F929F92AF92BF92CF92DF92D6
:10374000EF92FF920F931F93DF93CF930F92CDB71A
:10375000DEB75C01062F81E490E049830E943E2998
:10376000D82EC92EE82EF92EF701E05CFF4F4981D3
:10377000408310E040E050E01FC02815390554F4A4
:10378000241735073CF0D501A80FB11D9C919083FB
:103790008F5F01C010822F5F3F4F3196203431057B
:1037A00061F7C801B7010E94CD0C0F5F1F4F80E485
:1037B0008816910469F0A40188E0882E912C840E6B
:1037C000951EC601E92FFC2D20E030E080E0D5CF2A
:1037D000C7010E94D8290F90CF91DF911F910F91BF
:1037E000FF90EF90DF90CF90BF90AF909F908F9021
:1037F00008951F93CF93DF93162FC82FD92F07C09B
:103800000E941E1C612F41E00E949A1B185F899143
:103810008823B1F70E94780DEC01FC01E05CFF4FBA
:103820008AE08083812F90E0BE010E94CD0CCE0102
:103830000E94D829DF91CF911F910895982F90521F
:103840009F3538F08D3011F08A3011F481E201C0DB
:103850008FE38052E82FF0E083E0EE0FFF1F8A95A0
:10386000E1F7EE52FA4FA3EDB2E084918D933196D9
:1038700082E0AB3DB807C9F7CD0108970895A8E3EA
:10388000B0E0E5E4FCE10C94072929833A834B83FB
:103890005C836D837E838F839887A986BA86CB8667
:1038A000DC86ED86FE860F87188BE984FA840B850B
:1038B0001C852D853E854F85588929803A804B800F
:1038C0005C802DA23EA24FA258A6AD80BE80CF80C4
:1038D000D884211531054105510509F0A6C3AE1460
:1038E000BF04C006D10608F03FC120E0E21620E088
:1038F000F20621E0020720E0120758F43FEFE3163A
:10390000F1040105110509F090F420E030E0A9016F
:1039100017C040E0E41640E0F40640E0040741E050
:10392000140750F420E130E040E050E009C028E006
:1039300030E040E050E004C028E130E040E050E0FA
:10394000D801C701022E04C0B695A7959795879513
:103950000A94D2F780539F4FDC016C9180E290E093
:10396000A0E0B0E0821B930BA40BB50B861B910962
:10397000A109B1090097A105B105A1F1082E04C064
:10398000EE0CFF1C001F111F0A94D2F7A60195012F
:10399000082E04C0220F331F441F551F0A94D2F76C
:1039A00060E270E0681B790BADA0BEA0CFA0D8A4E8
:1039B00004C0D694C794B794A7946A95D2F7A22A64
:1039C000B32AC42AD52A2DA03EA04FA058A404C0D3
:1039D000220C331C441C551C8A95D2F72DA23EA202
:1039E0004FA258A6380188249924A8019701407055
:1039F0005070298F3A8F4B8F5C8FC601B501A4019F
:103A000093010E94E528222E532E442E352E6D8FD1
:103A10007E8F8F8F98A3C601B501A40193010E94E8
:103A2000E528822D952DA42DB32D1C012D01C20159
:103A3000B101298D3A8D4B8D5C8D0E94C6285B01AA
:103A40006C014D8D5E8D6F8D78A1DA0199278827E5
:103A50004DA15EA16FA178A59B0144275527822B1C
:103A6000932BA42BB52B8A159B05AC05BD05E0F463
:103A7000089421083108410851088E0D9F1DA01F90
:103A8000B11F8E159F05A007B10770F08A159B0521
:103A9000AC05BD0548F408942108310841085108D7
:103AA0008E0D9F1DA01FB11F9C01AD012A193B095E
:103AB0004C095D0959016A01CA01B901A4019301C8
:103AC0000E94E52829A739A349AB5DA76D8F7E8F9A
:103AD0008F8F98A3C601B501A40193010E94E52828
:103AE000A9A4B9A0C9A8DDA4C601B501298D3A8D44
:103AF0004B8D5C8D0E94C6283B014C016D8D7E8DE7
:103B00008F8D98A1AB01332722278DA19EA1AFA154
:103B1000B8A5A070B070282B392B4A2B5B2B26152B
:103B2000370548055905C0F40894A108B108C10833
:103B3000D1082E0D3F1D401F511F2E153F05400778
:103B4000510750F0261537054805590528F4089403
:103B5000A108B108C108D1088101FF24EE24EA2898
:103B6000FB280C291D29A1C4E114F104010511054C
:103B700059F461E070E080E090E0A80197010E94B4
:103B8000E52879018A0110C070E0E71670E0F706B9
:103B900071E0070770E0170758F48FEFE816F1049B
:103BA0000105110509F090F420E030E0A90117C0EB
:103BB00090E0E91690E0F90690E0090791E0190716
:103BC00050F420E130E040E050E009C028E030E06F
:103BD00040E050E004C028E130E040E050E0D8018F
:103BE000C701022E04C0B695A795979587950A94AC
:103BF000D2F780539F4FDC018C91280F311D411D5E
:103C0000511D80E290E0A0E0B0E0821B930BA40B7A
:103C1000B50B61F4150126012E183F08400A510A20
:103C200081E0A82EB12CC12CD12C23C1082E04C0B8
:103C3000EE0CFF1C001F111F0A94D2F7150126017C
:103C4000022E04C056944794379427940A94D2F7CE
:103C500035014601082E04C0660C771C881C991C8F
:103C60000A94D2F76D8E7E8E8F8E98A28DA09EA024
:103C7000AFA0B8A404C0B694A794979487942A954B
:103C8000D2F7A5019401AD8CBE8CCF8CD8A0A22A0E
:103C9000B32AC42AD52AAD8EBE8ECF8ED8A22DA12E
:103CA0003EA14FA158A504C0220F331F441F551F2A
:103CB0008A95D2F72DA33EA34FA358A73801882495
:103CC0009924B801A7016070707049A75AA76BA723
:103CD0007CA7C201B101A40193010E94E528298FAC
:103CE00039AB4DA75DAB69A37AA38BA39CA3C2019B
:103CF000B101A40193010E94E528A98CB9A8CDA423
:103D0000DDA8A98EBA8ECB8EDC8EC601B50129A5A1
:103D10003AA54BA55CA50E94C6285B016C0129A0B1
:103D20003AA04BA05CA0D101992788272D8C3E8C0E
:103D30004F8C58A0920144275527822B932BA42BFC
:103D4000B52B8A159B05AC05BD0530F5298D3A8D3F
:103D50004B8D5C8D2150304040405040298F3A8F30
:103D60004B8F5C8F8E0D9F1DA01FB11F8E159F0561
:103D7000A007B10788F08A159B05AC05BD0560F466
:103D80002150304040405040298F3A8F4B8F5C8FFC
:103D90008E0D9F1DA01FB11FAC01BD014A195B090B
:103DA0006C097D095A016B01CB01BA01A401930191
:103DB0000E94E528522E432E342E252E69A37AA385
:103DC0008BA39CA3C601B501A40193010E94E52821
:103DD000652C742C832C922CC401B30129A53AA51F
:103DE0004BA55CA50E94C6289B01AC0169A17AA1E4
:103DF0008BA19CA16B01BB24AA248D8D9E8DAF8DC0
:103E0000B8A1A070B070A82AB92ACA2ADB2AA216C3
:103E1000B306C406D506E0F4089461087108810869
:103E20009108AE0CBF1CC01ED11EAE14BF04C0064C
:103E3000D10670F0A216B306C406D50648F408945D
:103E40006108710881089108AE0CBF1CC01ED11E0C
:103E500015012601221A330A440A550A898D9A8DC2
:103E6000AB8DBC8D6C01BB24AA24A628B728C8281A
:103E7000D9283801882499246D8E7E8E8F8E98A241
:103E8000A80197014070507029A73AA74BA75CA7DB
:103E9000C201B101A40193010E94E528922E832E54
:103EA000742E652E69A37AA38BA39CA3C201B101D2
:103EB0002D8D3E8D4F8D58A10E94E528892D982D7E
:103EC000A72DB62D898F9A8FAB8FBC8FBC01CD01EA
:103ED00029A53AA54BA55CA50E94C6283B014C012B
:103EE00049A15AA16BA17CA1DA01992788272DA0AD
:103EF0003EA04FA058A4920144275527822B932B14
:103F0000A42BB52B86159705A805B90530F5298D85
:103F10003A8D4B8D5C8D2150304040405040298F70
:103F20003A8F4B8F5C8F8E0D9F1DA01FB11F8E157A
:103F30009F05A007B10788F086159705A805B90564
:103F400060F42150304040405040298F3A8F4B8FD1
:103F50005C8F8E0D9F1DA01FB11FAC01BD014619C6
:103F60005709680979093A014B01CB01BA012D8D36
:103F70003E8D4F8D58A10E94E528522E432E342E9F
:103F8000252E69A37AA38BA39CA3C401B3012D8D15
:103F90003E8D4F8D58A10E94E528652C742C832CF2
:103FA000922CC401B30129A53AA54BA55CA50E949A
:103FB000C6281B012C0169A17AA18BA19CA1AB0190
:103FC000332722278DA19EA1AFA1B8A5A070B07004
:103FD000282B392B4A2B5B2B22153305440555051D
:103FE000C0F4089461087108810891082E0D3F1DE6
:103FF000401F511F2E153F054007510750F0221555
:1040000033054405550528F40894610871088108B2
:104010009108898D9A8DAB8DBC8D8C01FF24EE2487
:10402000E628F7280829192943C2A216B306C406B0
:10403000D50608F42AC2203090E0390791E04907FC
:1040400090E0590750F42F3F31054105510509F023
:1040500090F466247724430119C02030A0E03A0789
:10406000A0E04A07A1E05A0760F490E1692E712CA4
:10407000812C912C0BC088E0682E712C812C912C06
:1040800005C0B8E16B2E712C812C912CDA01C9018D
:10409000062C04C0B695A795979587950A94D2F7F4
:1040A00080539F4FFC018081680E711C811C911C04
:1040B00080E290E0A0E0B0E086199709A809B9096C
:1040C00089F42A153B054C055D0508F4E5C12DA0D2
:1040D0003EA04FA058A42E143F044006510608F0FD
:1040E000DBC1D3C189A719012A0104C0220C331CEA
:1040F000441C551C8A95D2F7D801C701062C04C070
:10410000B695A795979587950A94D2F7282A392AC4
:104110004A2A5B2AA801970109A404C0220F331F71
:10412000441F551F0A94D2F729A33AA34BA35CA3BB
:1041300086017501062C04C016950795F794E7943F
:104140000A94D2F7B601A50109A404C0440F551F73
:10415000661F771F0A94D2F74D8F5E8F6F8F78A3FB
:104160006DA17EA18FA198A504C09695879577959E
:1041700067956A94D2F73B014C018D8D9E8DAF8D72
:10418000B8A186299729A829B9298D8F9E8FAF8F2D
:10419000B8A35201CC24DD24A201910140705070DB
:1041A00029AB3AAB4BAB5CABC801B701A60195019B
:1041B0000E94E528622E932E842E752E6DA77EA771
:1041C0008FA798ABC801B701A60195010E94E52809
:1041D000E62CF92C082D172DE98EFA8E0B8F1C8FEB
:1041E000C801B70129A93AA94BA95CA90E94C62810
:1041F0006DA47EA48FA498A88301FF24EE246D8C67
:104200007E8C8F8C98A0940144275527E22AF32AAC
:10421000042B152BE616F7060807190730F5298D2C
:104220003A8D4B8D5C8D2150304040405040298F5D
:104230003A8F4B8F5C8FE20CF31C041D151DE214AA
:10424000F3040405150588F0E616F70608071907B4
:1042500060F42150304040405040298F3A8F4B8FBE
:104260005C8FE20CF31C041D151DE61AF70A080BFF
:10427000190BC801B701A60195010E94E5282DABD5
:104280003EAB4FAB58AF6DA77EA78FA798ABC801C9
:10429000B701A60195010E94E5286DA87EA88FA808
:1042A00098ACC401B30129A93AA94BA95CA90E9401
:1042B000C6289B01AC01ADA4BEA4CFA4D8A8D5014B
:1042C00099278827AD8CBE8CCF8CD8A06FEFE62EB7
:1042D0006FEFF62E012D112DAE20BF20C022D1226E
:1042E0008A299B29AC29BD2982179307A407B50702
:1042F000E0F408946108710881089108820D931D0B
:10430000A41DB51D82159305A405B50570F082178F
:104310009307A407B50748F4089461087108810859
:104320009108820D931DA41DB51D1C012D01221A9B
:10433000330A440A550A2D8E3E8E4F8E58A2A98C00
:10434000BA8CCB8CDC8C8501FF24EE24E628F72880
:1043500008291929AFEFAA2EAFEFBA2EC12CD12C04
:10436000AE20BF20C022D12218014424552469A0C8
:104370007AA08BA09CA02FEF3FEF40E050E062229C
:1043800073228422952269A17AA18BA19CA1AC0100
:1043900066277727498F5A8F6B8F7C8FC601B501AF
:1043A000A40193010E94C62869A37AA38BA39CA3AE
:1043B000C601B501298D3A8D4B8D5C8D0E94C628B2
:1043C0005B016C01C201B101A40193010E94C628E6
:1043D0003B014C01C201B101298D3A8D4B8D5C8DA1
:1043E0000E94C6289B01AC01A60CB71CC81CD91C96
:1043F00029A03AA04BA05CA0C201AA27BB27A80E07
:10440000B91ECA1EDB1EA614B704C804D90420F4C2
:10441000205030404F4F5F4FC601AA27BB27820F65
:10442000931FA41FB51F4D8C5E8C6F8C78A048160F
:1044300059066A067B0618F184159505A605B70589
:10444000A1F56501BB24AA2489A19AA1ABA1BCA1B5
:10445000A070B070A80EB91ECA1EDB1E8DA19EA151
:10446000AFA1B8A509A404C0880F991FAA1FBB1F3C
:104470000A94D2F78A159B05AC05BD05B0F40894E3
:10448000E108F1080109110910C0AA24BB24650143
:10449000EE24FF2487010CC0AA24BB24650181E01F
:1044A000E82EF12C012D112D03C0AA24BB24650197
:1044B000FE01719688E0DF011D928A95E9F7E98A8D
:1044C000FA8A0B8B1C8BAD8ABE8ACF8AD88E2E2D92
:1044D0003A894B895C896A2D7E898F89988DE89607
:1044E000E2E10C942329ACE3B0E0E9E7F2E20C94BA
:1044F0000729F82FE92FA986BA86CB86DC86ED86B8
:10450000FE860F87188BE984FA840B851C858D85C0
:104510009E85AF85B889298F3A8F4B8F5C8F298C08
:104520003A8C4B8C5C8C2DA23EA24FA258A63B012C
:104530008F2E9E2E130124010097A105B10509F0CD
:104540000DC36E147F048006910608F0F7C020E0CA
:10455000E21620E0F20621E0020720E0120758F4FC
:104560003FEFE316F1040105110509F090F480E036
:1045700090E0DC0117C040E0E41640E0F40640E0C3
:10458000040741E0140750F480E190E0A0E0B0E0BF
:1045900009C088E090E0A0E0B0E004C088E190E0CD
:1045A000A0E0B0E0A8019701082E04C056954795F9
:1045B000379527950A94D2F720533F4FF901208170
:1045C000F0E2AF2EB12CC12CD12CA81AB90ACA0A1C
:1045D000DB0AA21AB108C108D108AD8EBE8ECF8EFB
:1045E000D8A2A114B104C104D10499F12D8D022ED9
:1045F00004C0EE0CFF1C001F111F0A94D2F7022EFC
:1046000004C0660C771C881C991C0A94D2F760E2DF
:1046100070E06A197B09298C3A8C4B8C5C8C04C045
:1046200056944794379427946A95D2F726283728CA
:1046300048285928498D5A8D6B8D7C8D04C0440FB4
:10464000551F661F771F2A95D2F74DA35EA36FA350
:1046500078A7380188249924C801B7018070907028
:10466000698F7A8F8B8F9C8FC201B101A401930156
:104670000E94E528D22EA32EC42EB52E69A37AA3BC
:104680008BA39CA3C201B101A40193010E94E52860
:104690006D2D7A2D8C2D9B2D298D3A8D4B8D5C8D1A
:1046A0000E94C6285B016C0129A03AA04BA05CA027
:1046B000D101992788272DA03EA04FA058A4920190
:1046C00044275527822B932BA42BB52B8A159B05AA
:1046D000AC05BD0590F48E0D9F1DA01FB11F8E155A
:1046E0009F05A007B10748F08A159B05AC05BD05DD
:1046F00020F48E0D9F1DA01FB11F9C01AD012A1932
:104700003B094C095D0959016A01CA01B901A401BB
:1047100093010E94E528522E232E442E352E69A3A4
:104720007AA38BA39CA3C601B501A40193010E94A7
:10473000E528652D722D842D932DC5C1E114F1045A
:104740000105110559F461E070E080E090E0A801F6
:1047500097010E94E52879018A0110C050E0E51612
:1047600050E0F50651E0050750E0150758F46FEFEB
:10477000E616F1040105110509F090F480E090E0DF
:10478000DC0117C070E0E71670E0F70670E007077D
:1047900071E0170750F480E190E0A0E0B0E009C0BC
:1047A00088E090E0A0E0B0E004C088E190E0A0E004
:1047B000B0E0A8019701082E04C05695479537959B
:1047C00027950A94D2F720533F4FF9012081820F99
:1047D000911DA11DB11D50E2252E312C412C512CD3
:1047E000281A390A4A0A5B0A2D8E3E8E4F8E58A22D
:1047F000211431044104510439F464015301AE1809
:10480000BF08C00AD10AEBC02D8D022E04C0EE0CE9
:10481000FF1C001F111F0A94D2F713012401082E58
:1048200004C056944794379427940A94D2F76401AD
:104830005301022E04C0AA0CBB1CCC1CDD1C0A9424
:10484000D2F7498D5A8D6B8D7C8D04C07695679516
:10485000579547958A95D2F7A42AB52AC62AD72A0A
:10486000A9A2BAA2CBA2DCA2698D7A8D8B8D9C8D78
:1048700004C0660F771F881F991F2A95D2F76DA372
:104880007EA38FA398A7380188249924D801C70153
:10489000A070B070898F9A8FAB8FBC8FC201B101AD
:1048A000A40193010E94E528D22EA32EC42EB52E7A
:1048B00069A77AA78BA79CA7C201B101A4019301A4
:1048C0000E94E5286D2D7A2D8C2D9B2D298D3A8DFA
:1048D0004B8D5C8D0E94C6285B016C0129A43AA413
:1048E0004BA45CA4D1019927882729A03AA04BA00A
:1048F0005CA0920144275527822B932BA42BB52B28
:104900008A159B05AC05BD0590F48E0D9F1DA01F5B
:10491000B11F8E159F05A007B10748F08A159B05AA
:10492000AC05BD0520F48E0D9F1DA01FB11F9C017D
:10493000AD012A193B094C095D0959016A01CA01F7
:10494000B901A40193010E94E528522E232E442E82
:10495000352E69A77AA78BA79CA7C601B501A4012C
:1049600093010E94E528652D722D842D932D298DAC
:104970003A8D4B8D5C8D0E94C6285B016C0149A568
:104980005AA56BA57CA5DA019927882729A13AA108
:104990004BA15CA140705070822B932BA42BB52BA4
:1049A0008A159B05AC05BD0590F48E0D9F1DA01FBB
:1049B000B11F8E159F05A007B10748F08A159B050A
:1049C000AC05BD0520F48E0D9F1DA01FB11F1C015D
:1049D0002D012A183B084C085D086201510118019D
:1049E00044245524A801970140705070298F3A8FB4
:1049F0004B8F5C8FC601B501A20191010E94E52891
:104A0000622E932E842E752E69A37AA38BA39CA36A
:104A1000C601B501A20191010E94E528662D792DFC
:104A2000882D972D298D3A8D4B8D5C8D0E94C6283F
:104A30005B016C0149A15AA16BA17CA1DA01992704
:104A400088276DA07EA08FA098A4940144275527A5
:104A5000822B932BA42BB52B8A159B05AC05BD058A
:104A600090F48E0D9F1DA01FB11F8E159F05A007EE
:104A7000B10748F08A159B05AC05BD0520F48E0DE5
:104A80009F1DA01FB11F9C01AD012A193B094C09B4
:104A90005D0959016A01CA01B901A20191010E948F
:104AA000E528622E932E842E752E69A37AA38BA3FC
:104AB0009CA3C601B501A20191010E94E528662DC3
:104AC000792D882D972D298D3A8D4B8D5C8D0E94E7
:104AD000C6285B016C0149A15AA16BA17CA1DA0136
:104AE000992788272DA13EA14FA158A5407050704D
:104AF000822B932BA42BB52B8A159B05AC05BD05EA
:104B000090F48E0D9F1DA01FB11F8E159F05A0074D
:104B1000B10748F08A159B05AC05BD0520F48E0D44
:104B20009F1DA01FB11F8A199B09AC09BD099C01DB
:104B3000AD010D8C04C056954795379527950A947D
:104B4000D2F7298B3A8B4B8B5C8B1D8A1E8A1F8A6E
:104B5000188E3A894B895C8960E0DEC26816790656
:104B60008A069B0618F48F2F9E2FD9C2803050E002
:104B7000950751E0A50750E0B50750F48F3F910528
:104B8000A105B10509F090F4AA24BB24650119C060
:104B9000803060E0960760E0A60761E0B60760F449
:104BA00040E1A42EB12CC12CD12C0BC038E0A32E97
:104BB000B12CC12CD12C05C028E1A22EB12CC12CC6
:104BC000D12C9C01AD010A2C04C056954795379510
:104BD00027950A94D2F720533F4FF9012081A20E66
:104BE000B11CC11CD11C20E230E040E050E02A1989
:104BF0003B094C095D0909F047C086159705A805D2
:104C0000B90548F0A98CBA8CCB8CDC8CAE14BF04EF
:104C1000C006D10638F1298D3A8D4B8D5C8D2E1949
:104C20003F09400B510B681A790A8A0A9B0AA1E0D6
:104C3000EA2EF12C012D112D698D7A8D8B8D9C8D95
:104C4000621773078407950718F0EE24FF24870185
:104C5000130124012E183F08400A510A2DA33EA338
:104C60004FA358A78DA19EA1AFA1B8A5898B9A8B00
:104C7000AB8BBC8B2D8A3E8A4F8A588E2DA13A89E8
:104C80004B895C89622D48C22DA31C012D01022E87
:104C900004C0220C331C441C551C0A94D2F7A9A64C
:104CA000D801C70104C0B695A79597958795AA9492
:104CB000D2F7282A392A4A2A5B2A2D8E3E8E4F8E19
:104CC00058A257016801022E04C0AA0CBB1CCC1CC0
:104CD000DD1C0A94D2F7ADA6BEA6CFA6D8AA1301B2
:104CE000240109A404C056944794379427940A9445
:104CF000D2F774016301022E04C0CC0CDD1CEE1C43
:104D0000FF1C0A94D2F7898D9A8DAB8DBC8D09A4B6
:104D100004C0B695A795979587950A94D2F7C82AA7
:104D2000D92AEA2AFB2AC9A2DAA2EBA2FCA2E98CC0
:104D3000FA8C0B8D1C8D04C0EE0CFF1C001F111F84
:104D40002A95D2F7E9AAFAAA0BAB1CAB0D8D1E8DE2
:104D50002F8D38A13901882499242070307009AF33
:104D60001AAF2BAF3CAFC201B101A40193010E9465
:104D7000E528A22ED32EE42E052F6DAB7EAB8FAB94
:104D800098AFC201B101A40193010E94E5288A2DC8
:104D90009D2DAE2DB02F898F9A8FAB8FBC8FBC010C
:104DA000CD0129AD3AAD4BAD5CAD0E94C6282DA911
:104DB0003EA94FA958AD8901FF24EE2429A03AA0AD
:104DC0004BA05CA0920144275527E22AF32A042B2A
:104DD000152BE616F7060807190750F5298D3A8DA9
:104DE0004B8D5C8D2150304040405040298F3A8F90
:104DF0004B8F5C8F2D8C3E8C4F8C58A0E20CF31C9B
:104E0000041D151DE214F3040405150588F0E616CB
:104E1000F7060807190760F4215030404040504021
:104E2000298F3A8F4B8F5C8FE20CF31C041D151DEC
:104E3000E61AF70A080B190BC801B701A401930180
:104E40000E94E528D22EC32EB42E552E6DAB7EAB1C
:104E50008FAB98AFC801B701A40193010E94E52868
:104E60008D2D9C2DAB2DB52D5C016D01C601B501BD
:104E700029AD3AAD4BAD5CAD0E94C6288B019C01BB
:104E80004DA85EA86FA878ACB2015527442789A128
:104E90009AA1ABA1BCA1A070B070482B592B6A2B72
:104EA0007B2B401751076207730700F50894A10890
:104EB000B108C108D1086D8C7E8C8F8C98A0460DEE
:104EC000571D681D791D461557056805790570F051
:104ED000401751076207730748F40894A108B10806
:104EE000C108D108460D571D681D791DDB01CA0197
:104EF000801B910BA20BB30B89A39AA3ABA3BCA3FA
:104F0000298C3A8C4B8C5C8CD101992788278A2973
:104F10009B29AC29BD292FEFE22E2FEFF22E012D78
:104F2000112DE822F9220A231B233D01882499240C
:104F3000ADA4BEA4CFA4D8A82FEF3FEF40E050E02F
:104F4000A222B322C422D5224DA55EA56FA578A9C1
:104F50001B0144245524C801B701A60195010E94F4
:104F6000C628698F7A8F8B8F9C8FC801B701A201E9
:104F700091010E94C6287B018C01C401B301A601E6
:104F800095010E94C6285B016C01C401B301A20116
:104F900091010E94C6289B01AC01EA0CFB1C0C1D70
:104FA0001D1D298C3A8C4B8C5C8CC201AA27BB2717
:104FB000E80EF91E0A1F1B1FEA14FB040C051D0551
:104FC00020F4205030404F4F5F4FC801AA27BB2725
:104FD000820F931FA41FB51F8701FF24EE24298D84
:104FE0003A8D4B8D5C8D40705070E20EF31E041FA5
:104FF000151F49A05AA06BA07CA0481659066A0646
:105000007B0670F084159505A605B70599F569A886
:105010007AA88BA89CA86E147F048006910650F590
:10502000A80197018DA49EA4AFA4B8A82819390996
:105030004A095B095C016D012D8C3E8C4F8C58A098
:10504000A218B308C408D50881E090E0A0E0B0E061
:10505000E216F3060407150718F080E090E0DC0183
:1050600025013601481A590A6A0A7B0AD301C2018E
:1050700079018A0169A87AA88BA89CA86E187F0874
:10508000800A910A9401830149A15AA16BA17CA1D4
:10509000481B590B6A0B7B0B81E090E0A0E0B0E06D
:1050A00089A89AA8ABA8BCA880169106A206B30648
:1050B00018F080E090E0DC01481B590B6A0B7B0B79
:1050C0005A016B0109A404C0AA0CBB1CCC1CDD1C3A
:1050D0000A94D2F70DA004C0369527951795079529
:1050E0000A94D2F7A02AB12AC22AD32AA98ABA8A54
:1050F000CB8ADC8ACB01BA010DA004C096958795B6
:10510000779567950A94D2F76D8B7E8B8F8B988FEE
:105110002A2D3A894B895C897E898F89988DEC96F6
:10512000E2E10C942329991B79E004C0991F96179A
:1051300008F0961B881F7A95C9F780950895AA1BD9
:10514000BB1B51E107C0AA1FBB1FA617B70710F072
:10515000A61BB70B881F991F5A95A9F780959095A4
:10516000BC01CD01089597FB092E07260AD077FDD3
:1051700004D0E5DF06D000201AF4709561957F4FCA
:105180000895F6F7909581959F4F0895629FD001FD
:10519000739FF001829FE00DF11D649FE00DF11DF2
:1051A000929FF00D839FF00D749FF00D659FF00DA1
:1051B0009927729FB00DE11DF91F639FB00DE11D8E
:1051C000F91FBD01CF0111240895A1E21A2EAA1BD7
:1051D000BB1BFD010DC0AA1FBB1FEE1FFF1FA217A7
:1051E000B307E407F50720F0A21BB30BE40BF50BA4
:1051F000661F771F881F991F1A9469F7609570952D
:10520000809590959B01AC01BD01CF0108952F922F
:105210003F924F925F926F927F928F929F92AF9246
:10522000BF92CF92DF92EF92FF920F931F93CF9393
:10523000DF93CDB7DEB7CA1BDB0B0FB6F894DEBF2A
:105240000FBECDBF09942A88398848885F846E8450
:105250007D848C849B84AA84B984C884DF80EE809A
:10526000FD800C811B81AA81B981CE0FD11D0FB6A3
:10527000F894DEBF0FBECDBFED010895CF93DF934D
:105280008230910510F482E090E0E091DD02F0912F
:10529000DE0240E050E020E030E026C06081718115
:1052A00068177907E0F06817790781F482819381A4
:1052B0002115310531F0D90113969C938E931297E5
:1052C0002BC09093DE028093DD0226C0411551056C
:1052D00019F06417750718F4AB01E901DF019F01AC
:1052E00072816381E72FF62F3097C1F64115510582
:1052F00001F1481B590B4430510580F412968D91F1
:105300009C911397209719F09B838A8304C09093F4
:10531000DE028093DD02FD01329646C0FD01E40FFE
:10532000F51F819391934250504011965C934E9398
:105330003BC02091DB023091DC022115310541F4A4
:105340002091D2013091D3013093DC022093DB0213
:105350002091D4013091D5012115310541F42DB7AB
:105360003EB74091D0015091D101241B350BE09103
:10537000DB02F091DC02E217F307A0F42E1B3F0BD7
:105380002817390778F0AC014E5F5F4F24173507B7
:1053900048F04E0F5F1F5093DC024093DB02819375
:1053A000919302C0E0E0F0E0CF01DF91CF9108954A
:1053B000CF93DF93009709F491C0FC0132971382D9
:1053C00012826091DD027091DE026115710581F437
:1053D00020813181280F391F8091DB029091DC02FE
:1053E0008217930799F5F093DC02E093DB0276C015
:1053F000DB0180E090E002C0CD01D901AE17BF070C
:1054000048F412962D913C91139721153105A1F77F
:10541000CD0121C0B383A283EF01499159919E012F
:10542000240F351FA217B30779F42D913C911197E2
:10543000240F351F2E5F3F4F3183208312962D910D
:105440003C91139733832283009729F4F093DE0273
:10545000E093DD0243C0DC011396FC93EE931297B8
:105460004D915D91A40FB51FEA17FB0769F42081E8
:105470003181240F351F2E5F3F4FEC013983288384
:10548000228133813B832A83E0E0F0E002C0FB010C
:10549000BC01DB0112968D919C9113970097B9F78F
:1054A0009B012E5F3F4F8D919C911197820F931F0F
:1054B0004091DB025091DC024817590779F430978C
:1054C00029F41092DE021092DD0202C013821282D1
:1054D000225030403093DC022093DB02DF91CF91E9
:1054E0000895A0E0B0E0E7E7FAE20C940F29EC01A0
:1054F000688179818A819B8161157105810591059A
:1055000021F464E279ED8BE597E02DE133EF41E0A2
:1055100050E00E944A2C79018A0127EA31E440E0F8
:1055200050E00E94C6285B016C01C801B7012CEE57
:1055300034EF4FEF5FEF0E94C6286A0D7B1D8C1D74
:105540009D1D97FF04C06150704080409048688363
:1055500079838A839B837F77CB01CDB7DEB7EAE07F
:105560000C942B290E94712A089586ED91E00E94E7
:10557000712A0895A0E0B0E08093D6019093D701FE
:10558000A093D801B093D90108952F923F924F92E2
:105590005F926F927F929F92AF92BF92CF92DF9273
:1055A000EF92FF920F931F93CF93DF933B01EA019A
:1055B0006115710519F0FB0180839183209739F003
:1055C0009E01225030402332310508F0D5C0C82E4C
:1055D000D92EF60111916F017F01812F90E00E9479
:1055E000D32B0097B1F71D3231F4F60111917F01F1
:1055F0009924939406C01B3219F4F60111917F018E
:105600009924209719F0C031D105D1F4103389F4D1
:10561000F7018081883711F0883559F4F70111813D
:1056200082E090E0E80EF91E92E0992AC0E1D0E015
:1056300007C0209729F41033B1F0CAE0D0E02BC0A6
:10564000CA30D10541F1C031D10521F0C830D105B2
:10565000A9F409C02FEFA22E2FEFB22E2FEFC22EEA
:105660002FE0D22E20C0C8E0D0E09FEFA92E9FEF00
:10567000B92E9FEFC92E9FE1D92E15C09E01442758
:1056800037FD4095542F6FEF7FEFCB010E94E52847
:1056900059016A0108C089E9A82E89E9B82E89E96B
:1056A000C82E89E1D82E60E020E030E0A9011E017B
:1056B000442437FC4094542C012F00530A3060F0EE
:1056C000812F81548A3110F4075006C0812F8156F2
:1056D0008A3150F5012F0755802F90E08C179D07D8
:1056E0001CF56F3FE9F0A216B306C406D506A8F074
:1056F000CA01B901A20191010E94C6289B01AC0117
:10570000802F90E0A0E0B0E0280F391F4A1F5B1FF8
:10571000281739074A075B0710F46FEF01C061E0F3
:10572000F70111917F01C8CF6114710481F06623E4
:1057300039F00894E108F108F301F182E08207C032
:1057400091FE05C0C7010297F3019183808390FE0B
:1057500007C050954095309521953F4F4F4F5F4F73
:1057600067FF0DC082E290E09093E0028093DF0239
:105770002FEF3FEFA90103C020E030E0A901B901FC
:10578000CA01DF91CF911F910F91FF90EF90DF90B1
:10579000CF90BF90AF909F907F906F905F904F9011
:1057A0003F902F900895911162C0803219F0895076
:1057B0008550D0F70895FB01DC0105900D92002083
:1057C000E1F70895FB019F01E8944230C4F04532AF
:1057D000B4F44A3029F497FB1EF4909581959F4FBD
:1057E000642F77270E949F28805D8A330CF0895DA3
:1057F0008193CB010097A1F716F45DE251931082DB
:10580000C9010C943A2CFA01CF93FF93EF93223005
:1058100044F1253234F5C22FE894CA3049F497FB9D
:105820003EF490958095709561957F4F8F4F9F4F77
:105830002C2F332744275527FF93EF930E94E52809
:10584000EF91FF91605D6A330CF0695D6193B9017E
:10585000CA01605070408040904051F716F4CDE28C
:10586000C19310828F919F91CF910C943A2C9927DC
:1058700088270895DC01FC01672F71917723E1F7F8
:10588000329704C07C916D9370836291AE17BF070D
:10589000C8F3089597FB092E05260ED057FD04D0B6
:1058A00094DC0AD0001C38F4509540953095219531
:1058B0003F4F4F4F5F4F0895F6F790958095709545
:0E58C00061957F4F8F4F9F4F0895F894FFCF53
:1058CE00202800290081422418182442810000005B
:1058DE0000000000000000000000000000814224D3
:1058EE001818244281814224181824428100000095
:1058FE0000000000000000000000000000814224B3
:10590E0018182442810101EE0E360FAA0E860F5092
:10591E000FCC0E140F020408101F3F7DFA3A200020
:10592E006D7300202800206D696E290073290A000E
:10593E000001020203030303040404040404040428
:10594E0005050505050505050505050505050505F9
:10595E0006060606060606060606060606060606D9
:10596E0006060606060606060606060606060606C9
:10597E0007070707070707070707070707070707A9
:10598E000707070707070707070707070707070799
:10599E000707070707070707070707070707070789
:1059AE000707070707070707070707070707070779
:1059BE000808080808080808080808080808080859
:1059CE000808080808080808080808080808080849
:1059DE000808080808080808080808080808080839
:1059EE000808080808080808080808080808080829
:1059FE000808080808080808080808080808080819
:105A0E000808080808080808080808080808080808
:105A1E0008080808080808080808080808080808F8
:105A2E0008080808080808080808080808080808E8
:0A5A3E002000E1020000010000005A
:00000001FF
